:020000040800F2
:1000000000000320E1110008A9110008AB1100084D
:10001000AD110008AF110008B11100080000000088
:10002000000000000000000000000000B311000804
:10003000B511000800000000B711000831120008D7
:100040003112000831120008311200083112000884
:100050003112000831120008311200083112000874
:100060003112000831120008311200083112000864
:100070003112000831120008311200083112000854
:100080003112000831120008311200083112000844
:100090003112000831120008311200083112000834
:1000A0003112000831120008311200083112000824
:1000B0003112000831120008311200083112000814
:1000C0003112000831120008311200083112000804
:1000D00031120008311200083112000831120008F4
:1000E00031120008311200083112000831120008E4
:1000F00031120008311200083112000831120008D4
:1001000031120008311200083112000831120008C3
:100110003112000831120008B9110008311200082C
:1001200031120008311200083112000831120008A3
:100130003112000831120008311200083112000893
:100140003112000831120008311200083112000883
:100150003112000831120008311200083112000873
:100160003112000831120008311200083112000863
:10017000311200083112000831120008000000009E
:100180003112000831120008311200083112000843
:100190003112000831120008311200083112000833
:0C01A00031120008311200083112000872
:1001AC0010B5054C237833B9044B13B10448AFF3A5
:1001BC0000800123237010BD0C0000200000000003
:1001CC008C12000808B5034B1BB103490348AFF36D
:1001DC00008008BD00000000100000208C120008F8
:1001EC0053B94AB9002908BF00281CBF4FF0FF3192
:1001FC004FF0FF3000F072B9ADF1080C6DE904CE90
:10020C0000F006F8DDF804E0DDE9022304B07047E5
:10021C002DE9F047089E04468846002B4BD18A42B4
:10022C00154667D9B2FA82F24AB1C2F1200701FA37
:10023C0002F320FA07F7954047EA030894404FEA87
:10024C00154E230CB8FBFEF71FFA85FC0EFB178826
:10025C0043EA084307FB0CF1994209D9EB1807F163
:10026C00FF3080F01B81994240F21881023F2B44F1
:10027C005B1AA4B2B3FBFEF00EFB103344EA03444A
:10028C0000FB0CFCA44509D92C1900F1FF3380F0BC
:10029C000781A44540F2048102382C4440EA07400F
:1002AC00A4EB0C0400271EB1D4400023C6E9004384
:1002BC003946BDE8F0878B4209D9002E00F0EB805F
:1002CC000027C6E9000138463946BDE8F087B3FA85
:1002DC0083F7002F47D18B4202D3824200F2FA807F
:1002EC00841A61EB030301209846002EE0D0C6E986
:1002FC000048DDE702B9FFDEB2FA82F2002A40F0D4
:10030C008F80491B4FEA154E1FFA85F80127B1FB68
:10031C00FEFC230C0EFB1C1143EA014308FB0CF101
:10032C00994207D9EB180CF1FF3002D2994200F236
:10033C00CD808446591AA3B2B1FBFEF00EFB10140B
:10034C0043EA044408FB00F8A04507D92C1900F136
:10035C00FF3302D2A04500F2B6801846A4EB080485
:10036C0040EA0C409FE7C7F1200CBB4022FA0CFE80
:10037C004EEA030E01FA07F420FA0CF521FA0CF3FD
:10038C004FEA1E482543B3FBF8F92C0C08FB193334
:10039C001FFA8EFA44EA034309FB0AF49C4202FA60
:1003AC0007F200FA07F10BD91EEB030309F1FF303A
:1003BC0080F087809C4240F28480A9F1020973444A
:1003CC001B1BADB2B3FBF8F008FB103345EA03443A
:1003DC0000FB0AFAA24508D91EEB040400F1FF3316
:1003EC006BD2A24569D90238744440EA0940A0FB9B
:1003FC000289A4EB0A044C45C2464B4654D351D057
:10040C00002E69D0B1EB0A0564EB030404FA0CFC72
:10041C00FD40FC404CEA0505C6E90054002747E7BF
:10042C00C2F1200320FA03F7954001FA02F021FAF9
:10043C0003F34FEA154E3843010CB3FBFEF71FFADA
:10044C0085F80EFB173341EA034107FB08F38B4297
:10045C0004FA02F407D9691807F1FF3C2FD28B423A
:10046C002DD9023F2944CB1A81B2B3FBFEF00EFB0F
:10047C00103341EA034100FB08F38B4207D969189A
:10048C0000F1FF3C17D28B4215D902382944C91A06
:10049C0040EA07473BE73746304609E70746E7E6B9
:1004AC001846FBE64145ABD2B8EB020A69EB0E02EB
:1004BC0001381346A4E76046E9E7184695E7674616
:1004CC00D1E781467CE702382C4447E7ACF1020CBB
:1004DC002B442FE7384608E73746E9E6704700BF5C
:1004EC0008B50B4B1A6842F400721A601A6842F491
:1004FC0080621A601A6842F480721A60032000F05D
:10050C002FF8002000F00CFE00F0EEFD002008BDDE
:10051C00003C0240034A044B11681B780B441360E7
:10052C00704700BF2800002000000020014B186815
:10053C00704700BF2800002038B50446FFF7F6FFCF
:10054C00631C1CBF054B1B78054618BFE418FFF74E
:10055C00EDFF401BA042FAD338BD00BF00000020C5
:10056C00074AD36823F4E0631B041B0C43F0BF63FE
:10057C00000243F4003300F4E0600343D36070479F
:10058C0000ED00E0174B70B5DC68C4F30224C4F135
:10059C000705042D04F1040328BF04254FF0FF3692
:1005AC00062B06FA05F38CBF033C002421EA030357
:1005BC00A34006FA04F422EA0404002843EA0403E4
:1005CC00A8BF00F160404FEA0313BCBF00F00F005E
:1005DC00054ADBB2AABF00F56140135480F8003322
:1005EC0070BD00BF00ED00E014ED00E0002808DB5A
:1005FC004209012300F01F0003FA00F0014B43F8FD
:10060C002200704700E100E02DE9F04F85B00B6847
:10061C00DFF8C4816E4ADFF8C491019300230124F2
:10062C00019D9C402540AC4240F0B8804C6824F0C1
:10063C00100C4FEA430E03260CF1FF3706FA0EF6A8
:10064C00012F6FEA060611D8876807EA060ACF68F9
:10065C0007FA0EF747EA0A078760476827EA050A90
:10066C00C4F300179F4047EA0A074760C76807EAC8
:10067C00060A8F6807FA0EF747EA0A07BCF1020F61
:10068C00C76016D14FEAD30A00EB8A0A03F0070BB6
:10069C00DAF820704FEA8B0B4FF00F0C0CFA0BFCB6
:1006AC0027EA0C0C0F6907FA0BF747EA0C07CAF894
:1006BC00207007683E4004F0030707FA0EFE4EEA6E
:1006CC0006060660E60069D54FF0000BCDF80CB0BD
:1006DC00D8F844703F4E47F48047C8F84470D8F8B7
:1006EC00447007F480470397039F23F0030707F137
:1006FC00804707F59C3703F0030ED7F808A04FEAA4
:10070C008E0E4FF00F0C0CFA0EFCB0422AEA0C0CB9
:10071C004BD006F58066B04249D006F58066B042F3
:10072C0047D006F58066B04245D006F58066B042EB
:10073C0043D0484543D006F50066B04241D006F59B
:10074C008066B0423FD006F58066B0423DD006F5DB
:10075C008066B04214BF0A26092606FA0EF646EA4F
:10076C000C06BE601668EF4314F4803F0CBF3E408D
:10077C002E431660566814F4003F0CBF3E402E43C7
:10078C005660966814F4801F0CBF3E402E43966052
:10079C00D668A40254BF3E402E43D6600133102BC2
:1007AC007FF43DAF05B0BDE8F08F5E46D5E701267E
:1007BC00D3E70226D1E70326CFE70426CDE70526AB
:1007CC00CBE70626C9E70726C7E70826C5E700BF1B
:1007DC00003C01400000024000380240001402407E
:1007EC000AB1816170470904FBE700002DE9F34170
:1007FC00044608B901203FE00368DD0710D42368E4
:10080C0098075AD423681A0700F19C8023685B0769
:10081C0000F1BA80A069002840F01B8100202BE079
:10082C00A74B9A6802F00C02042A07D09A6802F0CF
:10083C000C02082A0AD15B68590207D5A04B1B6829
:10084C009A03DCD56368002BD9D1D3E763689C4D40
:10085C00B3F5803F13D12B6843F480332B60FFF743
:10086C0065FE974D06462B689B03C8D4FFF75EFECA
:10087C00801B6428F7D9032002B0BDE8F081B3F5E2
:10088C00A02F04D12B6843F480232B60E3E72A6864
:10089C0022F480322A602A6822F480222A60002BFB
:1008AC00DDD1FFF743FE06462B689F03A7D5FFF764
:1008BC003DFE801B6428F7D9DDE7814B9A6812F066
:1008CC000C0F07D09A6802F00C02082A11D15B6851
:1008DC005E020ED47A4B1A68950702D5E268012A9B
:1008EC0088D11A68216922F0F80242EAC1021A6022
:1008FC0088E7E268734BB2B101221A60FFF716FE6B
:10090C006F4D06462B68980707D52B68226923F094
:10091C00F80343EAC2032B6074E7FFF707FE801B62
:10092C000228EFD9A7E71A60FFF700FE644D0646D0
:10093C002B6899077FF566AFFFF7F8FD801B02283F
:10094C00F6D998E76269604B7AB101221A60FFF719
:10095C00EDFD5B4D06466B6F9F073FF557AFFFF7FD
:10096C00E5FD801B0228F6D985E71A60FFF7DEFD4E
:10097C00534D06466B6F98077FF548AFFFF7D6FDD2
:10098C00801B0228F6D976E74D4B1A6C12F0805278
:10099C0028D101921A6C42F080521A641B6C03F03D
:1009AC0080530193019B0126484D2B68D9051BD51B
:1009BC00A368434D012B27D12B6F43F001032B6709
:1009CC00FFF7B4FD3E4D074641F288382B6F9B076D
:1009DC0039D5002E3FF41EAF394A136C23F08053E7
:1009EC00136417E70026DFE72B6843F480732B6052
:1009FC00FFF79CFD07462B68DA05D9D4FFF796FD67
:100A0C00C01B0228F7D936E7052B04D12B6F43F016
:100A1C0004032B67D0E72A6F22F001022A672A6FA2
:100A2C0022F004022A67002BCAD1FFF77FFD41F2A6
:100A3C00883807462B6F9807CBD5FFF777FDC01B7F
:100A4C004045F7D917E7FFF771FDC01B4045BDD9ED
:100A5C0011E71B4DAB6803F00C03082B47D01C4E61
:100A6C0000230228336035D1FFF760FD07462B6861
:100A7C0099011ED4D4E907321343626A43EA821304
:100A8C00E26A43EA0263A26A0D4C5208013A43EA55
:100A9C0002436B6001233360FFF748FD0546236872
:100AAC009A013FF5BBAEFFF741FD401B0228F6D97A
:100ABC00E1E6FFF73BFDC01B0228D8D9DBE600BFFF
:100ACC000038024000004742800E47420070004050
:100ADC0060004742FFF72AFD04462B689B017FF517
:100AEC009DAEFFF723FD001B0228F6D9C3E60128B3
:100AFC003FF4C2AE6868E36900F480029A427FF466
:100B0C0079AE226A00F03F0393427FF473AE626ABF
:100B1C0047F6C073034093427FF46CAEA26A00F4B4
:100B2C00403393427FF466AEE36A00F07060C01A03
:100B3C0018BF0120A0E600BF134908B58B6803F06D
:100B4C000C03042B03D0082B03D0104800E01048F2
:100B5C0008BD4A684B68496813F4800314BF0C48FD
:100B6C000A48C1F3881118BF002302F03F02A1FB11
:100B7C000001FFF735FB044B5B68C3F30143013302
:100B8C005B00B0FBF3F0E3E7003802400024F40014
:100B9C0000127A002DE9F0410D46044610B90120EF
:100BAC00BDE8F081434B1A6802F00F028A4228D349
:100BBC0021688F072DD4C80740D43E4B1A6802F029
:100BCC000F02AA4265D8226851076BD4130707D5C8
:100BDC00394A2169936823F4604343EAC103936063
:100BEC00FFF7AAFF344B354A9B68C3F30313D35C5E
:100BFC00D840334B1860334B186800F091FA002042
:100C0C00CEE7CAB21A701B6803F00F038B42C6D131
:100C1C00CEE7294B11F0040F1EBF9A6842F4E05244
:100C2C009A600E0742BF9A6842F460429A609A68D2
:100C3C00A06822F0F00202439A60BCE762681E4B87
:100C4C00012A1CD11B6813F4003FA8D01A4EB368BC
:100C5C0023F003031343B360FFF768FC41F28838B9
:100C6C000746B368626803F00C03B3EB820FA4D0A1
:100C7C00FFF75CFCC01B4045F3D9032090E7911EA5
:100C8C0001291B6802D813F0007FDEE713F0020F76
:100C9C00DBE7EAB21A701B6803F00F03AB427FF478
:100CAC007EAF90E70449E0688B6823F4E05303437C
:100CBC008B608BE7003C024000380240A412000815
:100CCC000800002004000020044B054A9B68C3F375
:100CDC008223D35C034A1068D84070470038024026
:100CEC00B4120008080000200F2303600B4B9A6815
:100CFC0002F0030242609A6802F0F00282609A6885
:100D0C0002F4E052C2609B68DB0803F4E053036119
:100D1C00034B1B6803F00F030B6070470038024055
:100D2C00003C024070470368DA6842F00102DA6066
:100D3C009A6802F00702062A1EBF1A6842F00102E6
:100D4C001A600020704770477047704770470368FF
:100D5C001A69910710B504460ED5DA6892070BD5BF
:100D6C006FF002021A619B6901229B07027777D010
:100D7C00FFF7EAFF0023237723681A69500710D581
:100D8C00DA6851070DD56FF004021A619B690222D3
:100D9C0013F4407F2277204668D0FFF7D5FF00235D
:100DAC00237723681A6912070FD5DA6810070CD558
:100DBC006FF008021A61DB6904229907227720463A
:100DCC005AD0FFF7C1FF0023237723681A69D20694
:100DDC0010D5DA68D0060DD56FF010021A61DB69F8
:100DEC00082213F4407F227720464BD0FFF7ACFF4C
:100DFC000023237723681A69D10708D5DA68D2074C
:100E0C0005D56FF001021A61204600F063F92368E2
:100E1C001A69100608D5DA68110605D56FF080023C
:100E2C001A61204600F0B7F823681A69520608D5F3
:100E3C00DA68500605D56FF040021A612046FFF7BC
:100E4C0085FF23681A69910622D5DA6892061FD5A8
:100E5C006FF0200220461A61BDE8104000F09AB8ED
:100E6C00FFF771FF2046FFF770FF83E7FFF76BFF7B
:100E7C002046FFF76AFF92E7FFF765FF2046FFF772
:100E8C0064FFA0E7FFF75FFF2046FFF75EFFAFE7C9
:100E9C0010BD0000304A0368904212D0B0F1804F70
:100EAC000FD0A2F57C4290420BD002F580629042AA
:100EBC0007D002F58062904203D002F5784290424E
:100ECC0019D14A6823F070031343234A904229D066
:100EDC00B0F1804F26D0A2F57C42904222D002F590
:100EEC00806290421ED002F5806290421AD002F5C8
:100EFC007842904216D0194A904213D002F5806283
:100F0C0090420FD002F5806290420BD0A2F598323D
:100F1C00904207D002F58062904203D002F58062C5
:100F2C00904203D1CA6823F4407313434A6923F0F7
:100F3C008003134303608B68C3620B688362064BA8
:100F4C00984203D003F58063984201D10B69036387
:100F5C0001234361704700BF000001400040014085
:100F6C0010B50446A0B190F83D3003F0FF021BB958
:100F7C0080F83C20FFF7D6FE022384F83D30206831
:100F8C00211DFFF787FF012384F83D30002010BDA1
:100F9C000120FCE77047704730B595B01022002156
:100FAC000AA800F065F90021142203A800F060F9EA
:100FBC0000241D4B01941A6C42F080521A641B6C75
:100FCC001A4A03F080530193019B0294136823F493
:100FDC00404343F480431360136803F4404302938B
:100FEC00029B01224FF48033CDE9082302254FF4F4
:100FFC0080036022CDE90E5308A80423CDE91032FA
:10100C00CDE91253FFF7F2FB0F23CDE903354FF473
:10101C00A0514FF48053CDE9061303A80321059486
:10102C00FFF7B8FD15B030BD00380240007000402D
:10103C0000B589B0FFF754FAFFF7AEFF1422002178
:10104C0003A800F015F90024204B00941A6B2048DB
:10105C0042F080021A631A6B02F080020092009A2E
:10106C0001941A6B42F001021A631A6B02F001022E
:10107C000192019A02941A6B42F040021A631B6BA4
:10108C0003F04003012202934FF4C041029B01255F
:10109C00FFF7A6FB4FF4C04303A90D48CDE9033578
:1010AC00CDE90544FFF7B0FA2A464FF40051084841
:1010BC00FFF796FB4FF47A70FFF73EFA22464FF497
:1010CC0000510348FFF78CFBFEE700BF00380240DD
:1010DC00001802400268034B9A4201D1FFF71ABA7A
:1010EC00704700BF0010004082B00C4B00210091F3
:1010FC005A6C42F480425A645A6C02F48042009258
:10110C00009A01911A6C42F080521A641B6C03F025
:10111C0080530193019B02B0704700BF003802401E
:10112C0030B5014689B000223620FFF72BFA362065
:10113C00FFF75CFA0025154B02951A6C144C42F023
:10114C0010021A641B6C03F01003029301A903A88C
:10115C00029BFFF7C9FDFFF7B7FD0E4B236040F272
:10116C00E733E36040000C4BB0FBF3F001386060F8
:10117C0020462561A560FFF7F3FE20B92046FFF756
:10118C00D2FD09B030BD0120FBE700BF00380240A2
:10119C002C0000200010004040420F007047FEE77A
:1011AC00FEE7FEE7FEE77047704770470148FFF720
:1011BC00CEBD00BF2C000020054BD3F8882042F494
:1011CC007002C3F888204FF000629A60704700BF2D
:1011DC0000ED00E0DFF834D0002103E00C4B5B584D
:1011EC00435004310B480C4B42189A42F6D30B4A2D
:1011FC0002E0002342F8043B094B9A42F9D3FFF773
:10120C00DBFF00F011F8FFF713FF7047000003201D
:10121C00CC120008000000200C0000200C00002064
:10122C006C000020FEE7000070B50D4E0D4CA41BA9
:10123C00A4100025A54209D10B4E0C4C00F020F84F
:10124C00A41BA4100025A54205D170BD56F825306D
:10125C0098470135EEE756F8253098470135F2E707
:10126C00C4120008C4120008C4120008C8120008F6
:10127C0002440346934200D1704703F8011BF9E77F
:10128C00F8B500BFF8BC08BC9E467047F8B500BF67
:08129C00F8BC08BC9E46704737
:1012A4000000000000000000010203040607080912
:0812B400000000000102030428
:0812BC0060EFFF7F010000005C
:0412C400D10100084C
:0412C800AD0100086C
:0C12CC0001000000100000000024F400ED
:04000005080011E1FD
:00000001FF
